:100000000AC0D0C03AC11895189589C1C7C11895C2
:100010001895189518958FED8DBFC0ECE8EB4E2E16
:10002000DD275D2EEEE7F0E0A0E6B0E088278D93B7
:100030003197E9F766248D9A8E9A8A988B988C98D6
:1000400085B7836085BF85B78C6085BF8BB78064BB
:100050008BBF8BB780688BBF80E08FBD84E08EBD87
:1000600085E083BF89B7826089BF789488EE93E08A
:10007000A0E68D939C9380E08093620080E0809363
:100080006300809164008F77809364000091620028
:10009000003009F003C09598969883C0013009F0AC
:1000A0000BC0959A96988AEF90E0CAD19598969A47
:1000B0008AEF90E0C5D175C0023009F00EC0959A64
:1000C00081E090E0BDD19598969A81E090E0B8D11A
:1000D00096988AEF90E0B4D164C0033009F00BC069
:1000E000959A81E090E0ACD19598969AA0E68D9192
:1000F0009C91A6D156C0043009F012C0959A9698EA
:100100008AEF90E09DD1969A8AEF90E099D19598E8
:100110008AEF90E095D196988AEF90E091D141C016
:10012000053009F003C0959A969A3BC0063009F055
:1001300010C0969A00916200063009F009C0959AA5
:1001400084E690E07DD1959884E690E079D1F2CF75
:1001500028C0073009F021C0959A84E190E070D161
:10016000959884E190E06CD1959A84E190E068D113
:10017000959888EC90E064D1969A84E190E060D103
:10018000969884E190E05CD1969A84E190E058D111
:10019000969888EE93E054D104C085E08093630084
:1001A00045D074CF0F921F922F923F924F925F9241
:1001B0007F92AF92BF920F931F932F933F934F93D2
:1001C0005F936F937F938F939F93AF93BF93CF93DF
:1001D000DF93EF93FF938FB78F9300916200073007
:1001E00009F004C080E08093620004C0A2E68C9114
:1001F0008F5F8C938F918FBFFF91EF91DF91CF91A4
:10020000BF91AF919F918F917F916F915F914F912E
:100210003F912F911F910F91BF90AF907F905F9072
:100220004F903F902F901F900F90189580E090E096
:10023000A5E68D939C93A3E64D915527A5E60D91D8
:100240001C91041715070CF401C013C0959A88EC93
:1002500090E0F6D0959888EC90E0F2D0A5E60D916C
:100260001C9141E050E0040F151FA5E60D931C936F
:10027000E2CF88EE93E0E4D008950F921F922F9280
:100280003F924F925F927F92AF92BF920F931F93D4
:100290002F933F934F935F936F937F938F939F938E
:1002A000AF93BF93CF93DF93EF93FF938FB78F936A
:1002B0000027A4E68C9187FB0EF401E040E00417D0
:1002C00009F009C089B7806889BF8091640080689F
:1002D0008093640008C089B78F7789BF80916400DC
:1002E0008F77809364008F918FBFFF91EF91DF91A3
:1002F000CF91BF91AF919F918F917F916F915F91BE
:100300004F913F912F911F910F91BF90AF907F9090
:100310005F904F903F902F901F900F9018950F92E5
:100320001F922F923F924F925F927F92AF92BF9215
:100330000F931F932F933F934F935F936F937F93ED
:100340008F939F93AF93BF93CF93DF93EF93FF93DD
:100350008FB78F938EEE95E89DBD8CBD82B390E4F0
:10036000892782BB8F918FBFFF91EF91DF91CF9152
:10037000BF91AF919F918F917F916F915F914F91BD
:100380003F912F911F910F91BF90AF907F905F9001
:100390004F903F902F901F900F9018950F921F92A3
:1003A0002F923F924F925F927F92AF92BF920F93A4
:1003B0001F932F933F934F935F936F937F938F93ED
:1003C0009F93AF93BF93CF93DF93EF93FF938FB739
:1003D0008F930027A0E38C9184FB0EF401E041E0B1
:1003E000041709F008C0959A969A84EF91E028D0F6
:1003F00080E0809362008F918FBFFF91EF91DF913A
:10040000CF91BF91AF919F918F917F916F915F91AC
:100410004F913F912F911F910F91BF90AF907F907F
:100420005F904F903F902F901F900F9018953197AD
:10043000F1F70895689462F80895E89462F80895D1
:10044000EF93FF93EE27E82BE92B31F0E0EDF7E097
:0E0450003197F1F70197D1F7FF91EF910895E1
:00000001FF
